:020000020000FC
:10000000A7CDAEC10000000020C0000093C00000DA
:1000100000009DC000000000000000000203040674
:10002000080C10182030406080000406080C1018DE
:100030002030406080A0C00000070F1F3F000D0D62
:1000400004050D050305030302004FB662FD0EC053
:10005000552009F00994C52DC095089483FDC795D6
:10006000C4BDC093A10064604FBE1895C0916400E8
:10007000089483FDC795C4BDC093A1006B7FC09158
:100080006400CF3F09F41FC070FF02C082FD05C0AD
:100090004FBEC098AC9895981895C098AC98959814
:1000A00075FD0DC065FD0BC0C9E0CA95F1F7C091A3
:1000B000B300C0FDAB9AC1FDAD9AC2FD949A2092E7
:1000C000A1004FBE189524BCCC27C064C8BF646093
:1000D000F6CFC1CF70FFBFCF65FDBDCFC09ABBCFFC
:1000E00070FFB9CF65FDB7CFAC9AB5CF70FFB3CF76
:1000F00065FDB1CF959AAFCFAB9870FFACCF65FDE2
:10010000AACFC7E0CA95F1F7C09AA5CFAD9870FF06
:10011000A2CF65FDA0CFC7E0CA95F1F7AC9A9BCFFF
:10012000949870FF98CF65FD96CFC7E0CA95F1F718
:10013000959A91CF4FB6C9B7CF7EC9BF6E7FCCB568
:10014000CE0DDDB5DF1DDBBDCABD4FBE18953FB678
:100150008F7EABB7A074A2118061A0E0ABBFA9B73E
:10016000AE7FA9BF7894A0916800AA2341F085FDD5
:100170002AC0A0916800AA95A093680024C040E01E
:1001800050E085FD14C0A0B396FDA095A2FD4FEFF1
:10019000A3E096FDA2E0A5BFAA27A064AABF8D7F19
:1001A000A0B396FDA095A2FD5FEF451741F7A8E12A
:1001B00061FDA093680085FD03C0A8E1A0936800DD
:1001C00040939700816085FD0EC0A0916900AA232D
:1001D00031F0A0916900AA95A093690004C08061E4
:1001E000AA27A064AABF80FF37C0A09197004A2F1A
:1001F00061FF8E7F85FD1CC0A091B600A430C1F4C4
:10020000403F08F040EFA42FA295AF704A0F5091E5
:10021000B800533069F0A695A69550FD01C0A6958B
:1002200052FD03C0A41B4A2F03C04A0F08F44FEF2E
:1002300040936100A72FA67079F0A0916D00A6955C
:10024000A69556E0A50F50916100A50FA0936100FF
:1002500018F4AFEFA09361004091B600443009F06C
:100260003EC0A0916100A093630040916300A09103
:100270009C004A1708F04A2FA0919E004A1708F0E8
:100280004A2F542EA091A200AA2309F422C0542F71
:100290005A1B10F4A42F50E0BA2E8894AA1FAA2E3D
:1002A000A091A400A095AA22A50E58F0A091A300A9
:1002B000A21509F0AA95AA0EA093A30048F04A2D12
:1002C00008C0A091A300BA1608F0A395A093A300BC
:1002D0004FEF409364007F7D485F08F07062A52D6A
:1002E000A03408F06860A0916000A395A09360001E
:1002F00051F0F894A9B7A160A9BF84FF02C0A0E49F
:10030000ABBF3FBE1895A0917400A395A093740055
:1003100041E050916800552329F085FF03C05A95AC
:1003200050936800A0919700A13018F020929A0095
:100330000DC020929B002092A500A0919A00AF5F73
:10034000A0939A0018F0AFEFA0939A00F894A9B781
:10035000A160A9BF84FF02C0A0E4ABBF3FBE189557
:100360003FB64CB55DB58F7EABB7A074A21180616E
:10037000A0E0ABBFA9B7AE7FA9BF789481FD23C031
:10038000A2E096FDA3E0A5BF8260A0B396FDA09574
:10039000A2FF05C040936500509366003CC1A3E0F6
:1003A00096FDA2E0A5BFAA27A064AABF8D7F85FF06
:1003B00001C024C140E0A0B396FDA095A2FD1EC1DE
:1003C000409397000DC1A3E096FDA2E0A5BF8D7FED
:1003D00061FF71C0A2E096FDA3E0A5BFAA27A064BB
:1003E000AABF82604093920050939300A090900027
:1003F0004A19B09091005B09BB24A22C4C385205DD
:1004000018F42092960049C0A091D600AA2359F171
:10041000483C520528F4A0E1BA2EAAE0AA2E23C037
:100420004836A1E05A0728F4A8E0BA2EAFE0AA2E79
:100430001AC0403DA2E05A0728F4A4E0BA2EAEE16B
:10044000AA2E11C0403AA5E05A0728F4A2E0BA2E1D
:10045000ACE3AA2E08C04839A8E05A0720F4A1E06E
:10046000BA2EA8E7AA2EC42EA0919400CA1AD52E9F
:10047000A0919500DA0ADD202AF4AFEFC094D09461
:10048000CA1ADA0A20929600A8E0A210A0E0CA14C4
:10049000DA0618F4A1E0A0939600409394005093DC
:1004A000950040919200509193004093900050939A
:1004B000910002E095C0A09165004A1BA0916600E2
:1004C0005A0B94FD80C093FD7EC092FD7AC086FFDA
:1004D00003C0D52EC42E0CC05695479591FD71C012
:1004E0005695479590FD6DC0D52EC42ED694C794D1
:1004F00061FD17C0AC2DAC51AD2DA24008F005C078
:10050000DD2079F4AC2DA85C60F4A0916700A39580
:10051000A0936700AA3008F471C020929700816010
:100520006DC0A0916700AA2319F0AA95A093670057
:10053000A22C5091BC0097FD06C0A090CA00533079
:1005400011F4A090D200AAEFAA0EA22DA21DCA18E3
:10055000DA0A4FB74170533049F4442321F087FD44
:1005600005C0806803C087FF01C08F77442359F01E
:10057000533031F4AFEFC094D094CA1ADA0A03C0F2
:1005800040E050E020C0533049F4CC0CDD1CAAE020
:10059000CA1AD20818F4A0E0CA2ED22CAFEFCA169D
:1005A000D20418F04FEF50E00EC0A091AE00CA9EEA
:1005B000412D000C441F50E008F012C04FEF50E0F6
:1005C0000FC05695479594FF07C0552309F04FEF8C
:1005D000A42FA6954A0F521D4F3F520508F04FEF2A
:1005E00040939700816061FF09C0AFE1A095A92306
:1005F000AB299A2F8F7DBB2009F48062A8E1A093DC
:10060000680085FF03C0AAE0A093680061FD03C0F5
:1006100085FD01C08F7E85FD03C0A6E0A093690023
:10062000F894A9B7A160A9BF84FF02C0A0E4ABBF42
:100630003FBE189511E00AC013E008C01AE006C0DA
:100640001EE104C014E602C018EC00C005E1BB279F
:10065000BA95F1F70A95D9F71A95C1F708952AE3E3
:1006600038E709C020E33CE806C02AE234EB03C0C7
:1006700025E238EC00C012E095FD9F7D95FF906269
:10068000BB27AD98BA95F1F7AC9ABA95F1F7AC984B
:10069000BA95F1F7AD9ABA95F1F7C09AB091AF005B
:1006A000BA95F1F7C098B7E8BA95F1F71A9521F71E
:1006B000022FB22FBA95F1F70A95D9F73A95D9F6E4
:1006C000AD980895221B39E0001F3A9509F408956A
:1006D000221F211B18F4210F8894F6CF0894F4CF21
:1006E000622C722CB0E08894B395221F331FE0F780
:1006F000379527958894912E802E020B130B10F4BA
:10070000192D082D10F4889401C00894661C771CDC
:10071000BA9571F7172D062D0895322D11232AF45D
:100720003A9500951095031B130BF894029F712CBA
:10073000002D129F912C802C7894780C172D921CF0
:10074000292DB4E06B2E2695179507956A94D9F755
:10075000332321F000951095031B130B089500918E
:10076000B6000430A1F1B0919700B15008F010C06C
:10077000B0916100B093630020927F0020928000CE
:100780002092810020928200209283006F7B1FC004
:100790006090B6006064B0916100B093620008E3BD
:1007A00017EC20917A0030917B0036952795B62D75
:1007B000BA9541F036952795B62DBA95BA9511F0B0
:1007C000369527958DDF00937F0010938000089564
:1007D00000917F00B09162000B1B10918000120904
:1007E00028F40038BFEF1B0740F009C00F3712058F
:1007F00008F405C00FE710E002C000E81FEF009307
:10080000840010938500089500918400B0918100C8
:100810000B0F10918500B09182001B1F20E03091DA
:10082000850033230AF42A95B09183002B1F1AF414
:10083000203F40F00AC02F3008F407C00FEF1FEF31
:100840002FE003C000E010E020EF30916300B09192
:100850009C003B1718F4323030F009C0B09185008D
:10086000BB235AF004C0B0918500BB2332F400933F
:100870008100109382002093830008952091D80076
:1008800000918400000F10918500111F46DF112395
:100890002AF40038BFEF1B0740F009C00F371205DC
:1008A00008F405C00FE710E002C000E81FEF0023C6
:1008B00052F0B0916200B01B0B2F18F0013008F01D
:1008C0000AC001E008C000950F5FB09162000B0FF5
:1008D00008F001C00FEF0093860008952091D90021
:1008E000009182001091830018DF11232AF4013057
:1008F000BFEF1B0740F009C00F3F120508F405C009
:100900000FEF10E002C001E01FEF112352F0B09191
:100910008600B01B0B2F18F0013008F00AC001E070
:1009200008C000950F5FB09186000B0F08F001C062
:100930000FEF0093630008950FEF677F71FD29C0EB
:1009400072FD09C06860B0917B00BA3020F0B52D0F
:10095000B03408F4677FB091D500BB23D1F0B091DB
:100960007B00BB23B1F00FEF10917B00ABDEF8945E
:10097000B091730072FDB5E00B9F112D002D78949E
:10098000112309F00FEFB0919F000B1710F40091A5
:100990009F0000939E00089500917A0010917B00C3
:1009A00000541140B0919E0010F4BA9501C0B39567
:1009B00011F0B0939E00089500C008952091B700F3
:1009C000B6B1B6FDFBCF04B115B1B6B1BF77B6B9BC
:1009D000B091AC00B395B093AC00B83060F1209208
:1009E000AC00B091D400BB2321F1112329F0B091C8
:1009F000AD00BF3F61F009C0B091AD000B1739F0F9
:100A000020F4BB2321F0BA9502C0B395E1F3009125
:100A10009C00B093AD00B13A50F400ECB43938F416
:100A200000E8B73820F400E4BA3708F400E0009397
:100A30009C00777F089510919C00B0E11B0F08F493
:100A40001FEF10939C00B091B600B43081F000917C
:100A50009C00B0916300B01B10F400916300B09152
:100A60009E000B1708F00B2F502E00936400B091DE
:100A7000AC00B73009F47860089502E3F894B091BF
:100A8000DA000B9F012D000C001F7894B0919C00A0
:100A90000B1710F000919C0000936100009363001D
:100AA000502E0093640000939F00089520927A00D6
:100AB000B0EFB0937B000895F8940CB51DB520916C
:100AC0007400789430917500609076000093750002
:100AD00010937600031B160971FD03C076FD81C0DB
:100AE0002BC070907700209377002709222311F004
:100AF0000FEF1FEF8090780090907900309378008E
:100B0000609279006918161910937C0000917500A5
:100B1000109176000819190920917A0030917B0014
:100B200036952795020F131F10F40FEF1FEF009358
:100B30007A0010937B0029C020917A0030917B00CD
:100B40003901B4E08B2EB2E09B2E343010F08A9441
:100B50009A94383010F08A949A94769467948A9490
:100B6000E1F726193709992021F0169507959A94EF
:100B7000E1F7200F311F20937A0030937B0028F497
:100B80003FEF30937A0030937B00323008F470648A
:100B900071FF02C0B3E00DC0B091C60000917100BA
:100BA000023838F0B395003A08F0B395B63008F043
:100BB000B5E09B2EB4E08B2E10917B0000917A0063
:100BC00024E0169507952A95E1F70819120928F0EF
:100BD000B02FB250B12FB20910F402E010E098012A
:100BE00026C020917A0030917B0039017694679479
:100BF0006694669466942619320906950695200F28
:100C0000321D20937A0030937B00323008F07F7BD6
:100C100004E0369527953695279526952695201B31
:100C200010F0223008F422E089019090C60060FDA7
:100C3000FECFE0908C00F0908D006160B9B7B0619C
:100C4000B9BF380176FD44C07694679400938C0058
:100C500010938D00B92DB330E1F0B0FD04C0060D46
:100C6000171D930106C0000F111F0250120922E048
:100C700030E0B92DB33068F020938E0030938F00B0
:100C8000009388001093890060928A0070928B0014
:100C90003DC000938E0010938F0020938800309306
:100CA000890060928A0070928B0071FF10C0B09131
:100CB0006D00B33060F000918F0010917C001595AD
:100CC000010F28F022F020928E0000938F001EC0AA
:100CD000669400938C00B92DB33091F0B0FD03C041
:100CE000060D262D03C0000F025022E0B92DB330AF
:100CF00038F020938E000093880060928A0006C02E
:100D000000938E002093880060928A0000917D00FD
:100D100002FD0350013029F495FD0AC0B0E0B7B9D7
:100D200009C0023019F4B7E0B7B904C095FDF6CF99
:100D3000B6E0B7B90091A400000F10F4BBE60B2792
:100D40000093A40060FDFECFB2E0B0936E0061603E
:100D5000B9B7B061B9BFB72FB670A1F020917A00D2
:100D600030917B0036952795F8940CB51DB5020F90
:100D7000131F1BBD0ABD6160B0E1B8BFB9B7B06158
:100D8000B9BF78940895606120927E0020E067FDED
:100D900020E206C0606120927E0020E267FD20E034
:100DA000789401E076FD11C0B72FB67009F06F7E20
:100DB000B0917B00B55048F002E0B55020F003E060
:100DC000B55008F006E071FD0AE060FD12C0B09178
:100DD0007E00BB2371F071FF08C0B0916D00B3308D
:100DE00020F0B0916E00BA9519F4789470615CC0EF
:100DF000AEDF789400000000F89476FD16C01091E4
:100E00007B00173008F017E0B5E01B0F72FD10E112
:100E100083FF110F62FF110F71FD12E8B4B56090EE
:100E2000A100B61990F2B10B80F2B0B7B77FB0BF96
:100E3000B8B1B0B7B860B0BFB0917E00B395B09311
:100E40007E00B8B176FD06C0B1E071FDB2E0BA95A2
:100E5000F1F7B8B1B072B21709F01BC071FF05C04D
:100E600003950A3008F00395B0CF64FF99CF6F7EE9
:100E70003CB56DB470907A0080907B00370D681C93
:100E80006BBC3ABD6160B0E1B8BFB9B7B061B9BF82
:100E900087CFB0916D00B23008F482CF64FD80CF6F
:100EA0000A9509F092CF7F7E20918E0030918F00BD
:100EB000F894B0E1B8BF0CB51DB5020F131F1BBDF0
:100EC0000ABDE0908800F09089006160B9B7B06118
:100ED000B9BF7894B72FB67039F0B0916D0072FF3A
:100EE000B395B0936D0009C074FF07C067FD05C0DE
:100EF00064FD03C0BF91BF91E3C4089500E063FFA8
:100F000003C064FF01C001E0F89410917100B7E0E4
:100F10001B9F212D102D7894200F2695179526952F
:100F200017952695179510937100183718F4B8E7A0
:100F3000B093710000917100B09172000B1720F016
:100F40006062C098AC98959860FDFECFE0908A00F2
:100F5000F0908B006160B9B7B061B9BF0895C49AD1
:100F6000B2E095FD07C0F894B0937D00AD98AB9AC0
:100F70007894EAC0F894B0937D00AD98949A7894F0
:100F8000E3C0C498B3E082FF24C095FD11C002E025
:100F9000F894B0937D00E6E8F0E00093B3009598F4
:100FA000949862FF02C0AC9A01C0AD9A7894CCC00C
:100FB00002E0F894B0937D00E6E8F0E00093B3001F
:100FC000C098AB9862FF02C0AC9A01C0AD9A789409
:100FD000BBC095FD0BC0F894B0937D00E0E7F0E056
:100FE000959862FF01C0AC9A7894AEC0F894B09323
:100FF0007D00E0E7F0E0C09862FF01C0AC9A789411
:10100000A3C0C49AB4E095FD07C0F894B0937D00E6
:10101000AB98949A789498C0F894B0937D00949883
:10102000AB9A789491C0C498B5E082FF24C095FD36
:1010300011C001E0F894B0937D00ECE7F0E000937C
:10104000B300AC98AD9862FF02C0C09A01C0AB9AE1
:1010500078947AC004E0F894B0937D00E0E9F0E081
:101060000093B300AC98AD9862FF02C0959A01C09E
:10107000949A789469C095FD0BC0F894B0937D0064
:10108000EAE6F0E0AC9862FF01C0C09A78945CC0D8
:10109000F894B0937D00E6E7F0E0AC9862FF01C001
:1010A000959A789451C0C49AB6E095FD07C0F8941B
:1010B000B0937D009498AD9A789446C0F894B0931C
:1010C0007D00AB98AD9A78943FC0C498B1E082FFA0
:1010D00024C095FD11C004E0F894B0937D00E0E9D0
:1010E000F0E00093B300C098AB9862FF02C0959AFD
:1010F00001C0949A789428C001E0F894B0937D00E0
:10110000ECE7F0E00093B3009598949862FF02C07A
:10111000C09A01C0AB9A789417C095FD0BC0F894A3
:10112000B0937D00E6E7F0E0C09862FF01C0959AB9
:1011300078940AC0F894B0937D00EAE6F0E09598C0
:1011400062FF01C0C09A78946F7D089529E630E06F
:10115000F9012092B300C098AC989598AB98AD98DF
:1011600094986B7F0895A4EBB0E009E00D9309E03B
:101170000D9304E00D930FEF0D9303E00D930FEF2C
:101180000D9309E00D9303E00D9301E00D9301E051
:101190000D93A0ECB0E001E00D930FEF0D930D93D4
:1011A0000D930D930D9303E00D930FEF0D930FEF40
:1011B0000D930D9305E20D9300ED0D9308E20D9351
:1011C00000E50D9304E00D930FEF0D9302E00D93F6
:1011D00000E00D930AE70D930FEF0D9300E00D93E0
:1011E00001E00D9300E00D9303E00D93089520912D
:1011F000BB008B7F233009F48460B091BC00B33016
:1012000019F09F7DB1FD90629F7BB091BD00B1FD53
:101210009064223011F0886001C0877F08950A959C
:10122000E00FF21DB4910895ECE1F0E00091B400FC
:10123000F6DFB093D800ECE1F0E00091B500EFDF0D
:10124000B093D900EAE2F0E00091BA00E8DFB09391
:10125000DA00B091D0000FEF1CE0B23011F400EAD8
:101260001AE0B33011F402E815E000937200109315
:101270007300E8E3F0E00091D700D1DFB093A20063
:10128000089508952091CA003091CB00B091BC0020
:10129000B33009F43E5097FF02C020E03FEFB32F78
:1012A000B21B6B2EB25810F4B2E86B2E00E003951F
:1012B000609EB12DBD57D8F30093AE00089590689D
:1012C000E1DFBED920E030E0B0E16B2EB5D9B091BE
:1012D00097002B0F321D6A94C9F7B4E03695279515
:1012E000BA95E1F7822E9F77CDDF0895F894E3E079
:1012F000F0E0B9E0B7BFB491B078C1F3F894A89525
:10130000B1B5B861B1BDB0E0B1BDB4E0BEBFBFE53D
:10131000BDBF1CDFB0E0B8BBB1E1B7BBB0E0B5BB4F
:10132000B8E3B4BBB0E0B2BBB0E3B1BB2224A0E0F1
:10133000B0E02D92AA31E9F7A0E6B0E00FEF2D92D0
:101340000A95E9F7B1E0B093A4000DDFE9D2B6B198
:10135000B460B6B90091CC000093AF00B1E0B09397
:101360006A00F89471D97BD96BD97CD969D97DD9B8
:1013700067D9F8940AEF1AEFA0B396FDA095A2FFE3
:101380001FC01A95C9F70A95B1F7E0E0FCE1B591E5
:10139000B43E39F4B591B03E21F4B591BF3F09F4A4
:1013A0000CC0E0E0F395F395B591B83F49F4B591E1
:1013B000B43931F4B591BA3A19F4EE27F695099497
:1013C00016DF32DF5EDF5EDF0091CC000093AF00FE
:1013D000BDDEB2E0B3BFB2E0BEBDB2E0B5BDB1E5C7
:1013E000B8BFB9BFB0B7B77FB0BFB8B1B0B7B8601A
:1013F000B0BF20D97894E0DAB3E096FDB2E0B5BF93
:10140000B0E4BBBFBB27B064BABF8D7F1DD962609B
:1014100033E02CE0B0919600BB2321F42CE03A9508
:1014200009F4A7CF0DD980FFA4CF8E7FB09197008C
:10143000B23078F3B92FBF710091990000939800F2
:10144000B0939900B01729F72A9521F76D7FB3E083
:1014500096FDB2E0B5BFBB27B064BABF8D7FB09137
:10146000D600BB2321F48062B92FB0709B2F8F7BF5
:1014700020926700E7D885FF05C0B0916700BA30B9
:1014800008F08064D9D802E085FF01C000E0B09187
:101490009700B017B8F3F894E2D8E1D8E0D8789480
:1014A000D3D820928700B091BC00B33009F474C047
:1014B000C3D8B091C000B13008F46EC0B0916A00DA
:1014C000B13008F469C085FD18C0B0919700BF3FE6
:1014D00008F462C0F894CCD87894B4D8B09197004E
:1014E000B130C0F7F894BBD8A9D8B9D87894AAD8A5
:1014F000B0919700BF3FB0F3D4C2B3E09B2E906889
:10150000F894C0DE78949ED8F8949F77BBDE8090E4
:101510009700B0919700BF37789408F445C08AD8F7
:10152000F894A6D878949A9451F7C9DEB82DB5509E
:10153000B093CB0089D8F89420D286D27894BAE0C0
:101540009B2E9068F8949EDE78947CD8F8949F77D0
:1015500099DE80909700B0919700BF37789478F724
:1015600069D8F8947CD86AD87AD878949A9449F74C
:10157000A6DEB82DBB5FB093CA0066D8F894FDD143
:1015800072D278945FD8F8947DDE7894B091970009
:10159000BF3F08F498CF85C200919700B0918700B3
:1015A0000B1710F0009387004DD801E0B091BC00FC
:1015B000B35009F405E0B0919700B01708F073CF6D
:1015C000F89456D855D854D878943ED820926A00CA
:1015D00020926B0020926C00B0916B00B395B09399
:1015E0006B00BF3F69F5B0916C00B395B0936C0090
:1015F000B091CE0009E1BA9559F002E3BA9541F0F5
:101600000DE7BA9529F00AEFBA9511F020926C0017
:10161000B0916C00B017A0F0B0916C00BA95B09387
:101620006C00B4EBB0936B00B091CD00B093AF0001
:10163000F8941ED87894B091CC00B093AF0002D843
:10164000FDD7B0916800BB2319F485FF01C091CE8E
:1016500001E085FD01C006E0B0919700B01708F4E5
:10166000BBCFB091BC00B35009F0ECD7B09168008B
:10167000BB2309F47ECEF89469DD209261002092AC
:10168000620020926300522C209264002092A300FA
:101690007894B091B900BB0FB093A00020927F0066
:1016A000209280002092810020928200209283006C
:1016B0002092AC0060E070E020927100B8E0B0933E
:1016C000AC007860B7D7B2E073FDB1E0B7B9B6B19E
:1016D000B068B064B6B9B6B1B6FDFDCF04B115B10E
:1016E000B6B1BF77B6B9112309F00FEF0093AD0083
:1016F00065D9B8E0B093AC0078608090BB00B2E0F0
:10170000B093BB0074DD8092BB00F894BFEFB09340
:101710009C00B3D9B0916100B0939C00B0939D0040
:10172000B0939E007894B1E0B0936100B0936300F1
:101730005B2EB0936400B093A600B0919B00B09371
:10174000A500B091BC00B33019F49F7D87FD906275
:101750007160726020926D00A6DCB7DCA7D9ACD9AD
:10176000A5D9AAD9A3D906C0F89441DD78942092CE
:10177000AC00777F0FDBF3D7C1DBF1DB9DD903DB57
:1017800066FD26D876FFD8D876FD06D9B7DBF9DB1B
:1017900093D900DB66FD38D8B1DB33DC8DD9F3DAC1
:1017A00066FD6CD8ABDB3FDC87D9F4DA66FD96D8F2
:1017B000A5DB79DC81D9E7DAB2E073FDB1E0B7B936
:1017C000B6B1B068B064B6B999DB7FDC75D9F6D82C
:1017D00071FF26C067FD24C0B0919F00B0939C00AC
:1017E000B0939D00B0919B00B093A500B1E0B09381
:1017F000A60018E12CE0B0916D00B11758F07D7F84
:10180000746020936F00B0919F00B0939C00B093E0
:101810009E0006C0B0919700B13008F0ABCF5AC01F
:1018200072FF10C067FD0EC0B0916F00BA9511F441
:101830007B7F9ACFB0936F00B0919700B13008F0E2
:1018400099CF48C020927000B0919A000AEFB0176B
:1018500008F040C085FF04C0B0916800BB23D1F1FF
:10186000B091BC00B33081F495FD03C087FD04C086
:101870000BC087FF01C008C067FD06C06068B0915B
:101880009F00B0939C008BCF00EF67FF05C0B09125
:101890009F00B0939C0000E2B0917B00B01708F469
:1018A00069CF67FF17C06F779F7D87FD9062746077
:1018B000B2E1B0936F00B0919F00B0939C005ACFFB
:1018C000B0917000B395B0937000B0919700BB23B6
:1018D00009F002C020927000F89438DC8090BB00C0
:1018E000B2E0B093BB0083DC8092BB002092610029
:1018F0002092620020926300522C20926400209279
:10190000A0007E7F789496D621DCB6B1B460B6B9DB
:1019100085FF05C0B0917000B53008F02ACD58CED3
:10192000EDE0F0E023D0053509F01BC0EEE0F0E07B
:101930001DD00A3A09F015C03AE0A4EBB0E0E3E0AC
:10194000F0E014D00D9331963A95D9F738E1A0EC38
:10195000B0E0EFE0F0E00AD00D9331963A95D9F778
:1019600002C001DC0AD0E7E2F0E00895E199FECF81
:10197000EEBBFFBBE09A0DB308951ED03AE0A4EB96
:10198000B0E0E3E0F0E00D910FD031963A95D9F751
:1019900038E1A0ECB0E0EFE0F0E00D9105D0319639
:1019A0003A95D9F712D00895E199FECF0DBBEEBB61
:1019B000FFBBE29AE19A0895EDE0F0E00FEFF4DF6B
:1019C000EEE0F0E00FEFF0DF0895EDE0F0E005E588
:1019D000EBDFEEE0F0E00AEAE7DF08953091B000D7
:1019E0000091B100313011F40093B400323011F4A1
:1019F0000093B500333011F40093B600343011F485
:101A00000093B800353011F40093BA00363011F469
:101A10000093C600373011F40093BB00383011F446
:101A20000093D700393011F40093D0003A3011F40C
:101A30000093BC003B3011F40093BD00089525E0F5
:101A400003D62A95E9F708950AD60CD60ED610D6F5
:101A5000F5D505D607D609D60BD6F0D500D602D6D1
:101A600004D606D6089504D600D6FCD5F8D5E6D51A
:101A7000FFD5FBD5F7D5F3D5E1D5FAD5F6D5F2D517
:101A8000EED508958090B0009090B100E8D5E7D5EC
:101A9000E6D5D4D58A94D1F7EBD5D0D59A94E1F791
:101AA0000895F894D1DF7894CADFC9DFB1E0B0932C
:101AB000B000B1E0B093B1002092B200F894E2DF40
:101AC0007894B5E06B2E70909700BED5B0919700DA
:101AD0007B16C9F7B13018F0BF3F40F107C07EDF79
:101AE000F8944BDFB1DFB8E0B1BDA9DF6A9459F7D4
:101AF000B091B200B395B093B200B33008F4DECF2A
:101B00009EDFB091B100B395B093B100F894B0915D
:101B1000B000BA95EEE3F0E0EB0FF21D049178947B
:101B20000395B091B100B01708F4C6CF88DF87DF06
:101B3000B091B000B395B093B000B091B000BC309C
:101B400008F4B7CF10DBF89418DFB8E0B1BD77DF49
:021B5000CDCBFB
:00000001FF
